S016000031313056636875616E67616E71692E7372656307
S3150800000000100020F9110008B9080008BB0800080C
S3150800001000000000000000000000000000000000D2
S31508000020000000000000000000000000BD080008F5
S315080000300000000000000000BF080008F1110008D9
S315080000404912000800000000491200084912000879
S315080000504912000849120008C1080008CB08000820
S3150800006000000000D5080008E5080008F5080008A3
S315080000700509000849120008491200080000000096
S3150800008049120008000000000000000015090008D9
S315080000900000000049120008491200084912000829
S315080000A000000000491200080000000025090008A9
S315080000B00000000000000000000000000000000032
S315080000C010B5064C2378002B07D1054B002B02D020
S315080000D0044800E000BF0123237010BD1000002073
S315080000E000000000C0370008044B10B5002B03D0F1
S315080000F00349044800E000BF10BDC04600000000E8
S3150800010014000020C037000802B4714649084900A7
S31508000110095649008E4402BC7047C04602B471466F
S3150800012049084900095C49008E4402BC7047C0462C
S31508000130002243088B4274D303098B425FD3030A18
S315080001408B4244D3030B8B4228D3030C8B420DD32B
S31508000150FF22090212BA030C8B4202D312120902B9
S3150800016065D0030B8B4219D300E0090AC30B8B42F7
S3150800017001D3CB03C01A5241830B8B4201D38B03A5
S31508000180C01A5241430B8B4201D34B03C01A52414A
S31508000190030B8B4201D30B03C01A5241C30A8B428D
S315080001A001D3CB02C01A5241830A8B4201D38B0278
S315080001B0C01A5241430A8B4201D34B02C01A52411C
S315080001C0030A8B4201D30B02C01A5241CDD2C3098E
S315080001D08B4201D3CB01C01A524183098B4201D30A
S315080001E08B01C01A524143098B4201D34B01C01AF5
S315080001F0524103098B4201D30B01C01A5241C3086D
S315080002008B4201D3CB00C01A524183088B4201D3DB
S315080002108B00C01A524143088B4201D34B00C01AC7
S315080002205241411A00D20146524110467047FFE733
S3150800023001B5002000F0F0F802BDC0460029F7D04D
S3150800024076E7704703460B437FD4002243088B4268
S3150800025074D303098B425FD3030A8B4244D3030B3F
S315080002608B4228D3030C8B420DD3FF22090212BA04
S31508000270030C8B4202D31212090265D0030B8B4280
S3150800028019D300E0090AC30B8B4201D3CB03C01A6A
S315080002905241830B8B4201D38B03C01A5241430B45
S315080002A08B4201D34B03C01A5241030B8B4201D335
S315080002B00B03C01A5241C30A8B4201D3CB02C01AA0
S315080002C05241830A8B4201D38B02C01A5241430A18
S315080002D08B4201D34B02C01A5241030A8B4201D307
S315080002E00B02C01A5241CDD2C3098B4201D3CB01AE
S315080002F0C01A524183098B4201D38B01C01A52415D
S3150800030043098B4201D34B01C01A524103098B4260
S3150800031001D30B01C01A5241C3088B4201D3CB004B
S31508000320C01A524183088B4201D38B00C01A52412E
S3150800033043088B4201D34B00C01A5241411A00D2DE
S3150800034001465241104670475DE0CA0F00D0494247
S31508000350031000D34042534000229C4603098B42B7
S315080003602DD3030A8B4212D3FC22890112BA030A3F
S315080003708B420CD3890192118B4208D389019211C1
S315080003808B4204D389013AD0921100E08909C30946
S315080003908B4201D3CB01C01A524183098B4201D348
S315080003A08B01C01A524143098B4201D34B01C01A33
S315080003B0524103098B4201D30B01C01A5241C308AB
S315080003C08B4201D3CB00C01A524183088B4201D31A
S315080003D08B00C01A5241D9D243088B4201D34B0035
S315080003E0C01A5241411A00D20146634652415B1077
S315080003F0104601D34042002B00D549427047634658
S315080004005B1000D3404201B5002000F005F802BD9C
S315080004100029F8D016E770477047C046D0400B0051
S31508000420D1409C46203AD3401843524263469340F3
S315080004301843704730B585B00C22002101A803F097
S31508000440B6F90422164C174B62618022236080237A
S315080004505202A261C2221B06012563600023FF32F5
S31508000460E2612000621DA360E36025612362D37701
S31508000470A56200F0E1FF002801D000F003FA80230E
S315080004805B0102930723200001A90195039301F05C
S31508000490C1F9002801D000F0F5F905B030BDC04615
S315080004A02C0000200024014030B5050089B0142234
S315080004B0002103A803F07BF9214B2A689A423CD114
S315080004C08020204B800099690143996180219A69AF
S315080004D0890202400192019A5A6990200A435A6198
S315080004E05B69C0050B400293029B022303A9039391
S315080004F00133049301F06CFC8022134C134BE26029
S31508000500921822618022D200236062610023202291
S3150800051020006360A360A261E36101F043FA00284A
S3150800052001D000F0AFF900220C2011002C6365629F
S3150800053001F0E8F90C2001F00FFA09B030BDC04609
S3150800054000240140001002406C0000200800024010
S3150800055013B50124104B21005A69092022435A6118
S315080005605B69002223400193019B01F0CBF9092026
S3150800057001F0F2F9210000220A2001F0C3F90A204D
S3150800058001F0EAF9002221000B2001F0BBF90B204B
S3150800059001F0E2F913BDC0460010024030B589B03B
S315080005A01422002103A803F002F980202F4BC00370
S315080005B059699025014359615A69ED050240802021
S315080005C00092009A596980020143596180215A694B
S315080005D0C90202400192019A5A6928000A435A61DF
S315080005E05B6901220B4002931021029B01F0ACFCCF
S315080005F000222800202101F0A7FC08230393C42326
S31508000600002428009B0303A90493059401F0E0FB4A
S3150800061030232800039303A92F3B049306930594DC
S3150800062001F0D6FB4023280003A9039304940594FC
S3150800063001F0CEFB80230393882328005B0303A9DC
S315080006400493059401F0C4FB22000221062001F060
S3150800065059F9062001F080F922002100072001F04F
S3150800066051F9072001F078F909B030BD00100240B1
S315080006700848094B10B5036006234360074BC3605F
S315080006809C239B00836001F079FC002801D000F0D0
S31508000690F9F810BDB000002000300040FF0F000040
S315080006A030B595B0282200210AA803F080F8102258
S315080006B00021684603F07BF81022002104A803F005
S315080006C076F80923089380235B021193802301247B
S315080006D002255B0308A809940F941095129301F05C
S315080006E087FC002801D072B6FEE707230290039024
S315080006F0210068460093019501F0ACFE002801D060
S3150800070072B6FEE7069004A8049401F037FF0028A5
S3150800071001D072B6FEE715B030BD0000F8B500F09E
S31508000720B9FDFFF7BDFFFFF739FFFFF711FFFFF729
S3150800073081FE00F0A3F9FFF79BFF00F065F9414B36
S3150800074041481988414A4B1E9BB283426FD8118093
S315080007503F4B19883F4B4A1E92B282426AD819808B
S315080007603D4C1B88226853633C4B3D4A19884B1CF9
S315080007709BB2012B62D911803A4E300001F030FC51
S31508000780200002F031F80021200002F0A3FA364CCE
S31508000790200002F02FFB20222000344902F0A4FF9B
S315080007A0334F344CFA223900200000F0EDFE902039
S315080007B000222021C00501F0C7FB3221002000F0ED
S315080007C0EDFCFA210120490000F0E8FC02202A4944
S315080007D000F0E4FC002000F0F7FC002809D0200017
S315080007E000F01CFF00F0EAF9FA223900200000F0B8
S315080007F0CBFE012000F0E8FC002807D0300001F00D
S31508000800EFFB90201021C00501F0A4FB022000F0A8
S31508000810DBFC002802D00222184B1A70184D2B78E0
S31508000820002BD7D000F0BCFB00232B70D2E70123A6
S3150800083013808DE7FA2292001A8091E70A23138023
S315080008409AE7C046003C0008FDFF0000140200209D
S31508000850023C00085A040020C0000020043C00089E
S315080008604C040020B0000020900100200A0400205B
S31508000870160200202C000020881300000400002027
S315080008807C04002072B6FEE701200A4B82B0996903
S315080008900143996180219A69490502400092009AAC
S315080008A0DA690A43DA61DB690B400193019B02B0FE
S315080008B07047C04600100240FEE7FEE770477047E3
S315080008C010B5082001F04EFB10BD10B5802001F0D0
S315080008D049FB10BD10B5024801F015F910BDC04618
S315080008E06C00002010B5024801F00DF910BDC04695
S315080008F00801002010B5024801F005F910BDC046F0
S315080009004C01002010B5024800F014FF10BDC04687
S315080009102C00002010B5024801F094FF10BDC04617
S31508000920C000002070B5114C200002F029FB1022EF
S315080009302368D969114218D01A62200002F05AFABF
S315080009400B4B0C4D1A78002A0AD10B4A0B48126831
S3150800095051682022521AD2B229001A7002F01EFFDC
S3150800096020222900200002F0BFFE70BD9001002061
S315080009707C0400200A040020080100205C040020F2
S315080009807047000007B50B4B02689A4211D18020C8
S31508000990094A4000D1690143D161D3690121034065
S315080009A00193ED380022019B00F0ACFF132000F004
S315080009B0D3FF07BD002000400010024010B5040018
S315080009C086B01422002101A802F0F1FE0B4B226822
S315080009D09A4210D180200A4AC002516901435161E6
S315080009E0536901A903400093009B0223054801931C
S315080009F0029301F0EDF906B010BDC0460020004094
S31508000A00001002400004004810B588B01C220021DE
S31508000A1001A802F0CCFE164C164B174A2360012398
S31508000A20636000232000A360E2602361A36101F0F4
S31508000A30EDFF002801D0FFF725FF200002F00EF891
S31508000A40002801D0FFF71EFF602300220193200033
S31508000A50CC3301A902930392059202F063F80028A9
S31508000A6001D0FFF70FFF2000FFF7A8FF08B010BD61
S31508000A70C000002000200040E70300000B480C4B94
S31508000A8010B5036096239B010C2243600023426144
S31508000A908360C36003618361C3610362436202F0DA
S31508000AA09DFD002801D0FFF7EDFE10BD9001002046
S31508000AB00038014030B5050089B01422002103A88A
S31508000AC002F075FE354B2A689A4265D18020344B70
S31508000AD0C00199690143996180219A698902024096
S31508000AE00192019A5A6990200A435A615B69C005C6
S31508000AF00B400293029BC023DB000393022304935B
S31508000B000133069303A9023B079301F061F9254CCB
S31508000B10254B8022236000236360A3602361636101
S31508000B20A361802320005B01E260E36100F03AFFE5
S31508000B30002801D0FFF7A6FE1C4B2C6765621C4CEB
S31508000B4080222360102363600023A360236163610E
S31508000B50A361802320005B01E260E36100F022FFCD
S31508000B60002801D0FFF78EFE8023124A9B001168E9
S31508000B701B200B4313600022EC661100656200F02F
S31508000B80C1FE1B2000F0E8FE10220B4B1B681968FB
S31508000B900A431A6050221A6209B030BD0038014073
S31508000BA000100240080100203000024044000240C4
S31508000BB04C010020000001409001002070B5294C2E
S31508000BC00121228813004800205A984242D8051C61
S31508000BD0904200D9151CAAB20131FA29F3D1991A03
S31508000BE0002904DD204908881B189B1A0B801F4C16
S31508000BF023785A1C2270032B2BD91B4D0521002361
S31508000C00E85EFFF71FFB03B219481A495843FFF776
S31508000C1019FB194B0A2100229B5E5843FFF712FB6A
S31508000C20164B174A1B785BB258430021535E00B235
S31508000C30C31AD9175B184B400A2B00DD1080114BDD
S31508000C401B78012B08D112880F4B1A8000232B80A2
S31508000C50237070BD0300BFE7002BF7D112880B4B3A
S31508000C60F3E7C046160200204A0400205704002075
S31508000C70E40C0000FF0F00004C04002005000020D3
S31508000C804E04002055040020520400205004002081
S31508000C9010B50400902001222021C00501F054F966
S31508000CA008490948A2B202F049F8084800F074FF5A
S31508000CB00128FAD1902000222021C00501F044F92C
S31508000CC010BDC0462A040020900100204C010020D7
S31508000CD07FB5414CA01C00F0F9F90600201D00F074
S31508000CE0F5F906210500200000F0F8F9020AD2B24B
S31508000CF0C0B2012E25D1022D22D1A17991421FD150
S31508000D00E27982421CD1354D237807212B7063780E
S31508000D1028006B700423AB70314B00229B5E1A12BD
S31508000D202B71304BEA701B785BB21A12AB716A7181
S31508000D3000F0D4F9030A28720B20EB71FFF7A8FF1D
S31508000D407FBDFF2E17D0022E29D0032EF8D1012DF4
S31508000D50F6D1A1799142F3D1E2798242F0D11F4DC1
S31508000D6023782B7063786B700223AB701E4B0022BE
S31508000D709B5E1A1224E0012DE2D1A1799142DFD1BE
S31508000D80E2798242DCD110221849684602F006FD53
S31508000D9010226946114802F001FD1120CEE7012D07
S31508000DA0CED1A1799142CBD1E2798242C8D10B4DFD
S31508000DB023782B706378AE706B700D4B1B881A0AFC
S31508000DC02B7105212800EA7000F088F9030AA8713A
S31508000DD06B710920B2E7C0465C0400202A04002093
S31508000DE04E040020040000204C040020F0370008C0
S31508000DF05A04002070B500230124174E86B00293CA
S31508000E0003930496059400F0EBFE694603A801AD2A
S31508000E1000F094FF002819D1104B31001B880330CD
S31508000E202B701B0A6B700E4B1B88AB701B0AEB7082
S31508000E300C4B00229B5E2B711B126B71019A029B55
S31508000E4000F016FF041E04D100F0DEFE200006B0F6
S31508000E5070BD0324FAE7C046003C000814020020CF
S31508000E605A0400204C040020F7B5444C65792079D3
S31508000E702D020543A01C00F029F906210090200048
S31508000E8000F02CF93E4F062201902100380002F0AE
S31508000E9085FC6A46019B10791B0A009A6DBADBB27B
S31508000EA0AEB2BB71F8710F2A28D1A2799A4214D131
S31508000EB0E379834211D1013EF62E14D8314B1D80B9
S31508000EC0012383F31088FFF795FF002805D180F3E7
S31508000ED0108823780A20002B2ED1202200212000FA
S31508000EE002F065FCF7BDFF2306213B717B712000EC
S31508000EF000F0F4F8030ABB71F871EAE7009A022ACF
S31508000F001DD1A2799A42E8D1E3798342E5D1FA2242
S31508000F10731E9BB292009342DFD21B4B1D801B4B64
S31508000F201B685E63012383F31088FFF763FF0028BD
S31508000F30D3D180F310880A30FFF7AAFECDE7009ACE
S31508000F40032ACAD1A2799A42C7D1E3798342C4D186
S31508000F500F4BF6180F4BB6B29E42BED828B20E4EAD
S31508000F600A25012807D00D4B68430021595EFFF773
S31508000F7069F93080D6E73580D4E7C0465C0400209E
S31508000F802A040020140200205A040020C000002071
S31508000F90E40C0000C81900004C0400204E04002090
S31508000FA010B50F4B0F491A7809880F4C91420FD18B
S31508000FB02278082A09D15B78032B04D0062B04D1A2
S31508000FC0FFF752FF01E0FFF783FE0023237010BDF1
S31508000FD0002AFAD12278082AF7D15B78EEE7C046CC
S31508000FE05C040020140200207C04002010B50400D4
S31508000FF080281DD190204021C00500F09FFF0128C0
S3150800100003D1284A137801331370274A137801331A
S31508001010DBB21370052B0AD9224B01211878022856
S3150800102000D802392148017000211170197010BDCD
S315080010300828FCD102201E4900F0B0F890202100B3
S31508001040C00500F07BFF1B4B012827D118701A4BEF
S3150800105000229B5E194A0021525E9B1A642B10DD02
S31508001060174A13780133DBB21370022BDFD900213C
S315080010701448017014480170FA2BD8D90323137049
S31508001080D5E7114A13780133DBB21370022BCED998
S315080010900C49087000200A490870EDE700221A700A
S315080010A0C5E7C04658040020540400200500002067
S315080010B08813000055040020520400205004002024
S315080010C059040020040000205604002002784078C5
S315080010D00002104340BA80B270470000FF22130096
S315080010E0F0B5084D084E094F013989B2A94202D117
S315080010F018021043F0BD047801305C40335D53405C
S315080011003A5DF1E7FFFF00000038000800390008E3
S315080011101C4A70B51368002B07D01368013B13608F
S31508001120002B02D10122184B1A7000220C25012629
S3150800113016482C0054430319596800290AD05968DF
S3150800114001395960002905D15E70215C012901D158
S31508001150996859600132042AEBD10D4B1A6801329D
S315080011601A6019680B4A914201D100221A600A4A8C
S3150800117013780133DBB2092B01D8137070BD002335
S31508001180FBE7C046BC040020B80400208804002001
S3150800119080040020FFFFFF7F84040020030030B591
S315080011A0032800D9FEE7012585F310880C200022C4
S315080011B05843044C2318596099605A70055582F3B0
S315080011C0108830BD8804002003000020032B09D8AE
S315080011D00C305843054B00221B185978C8B2012910
S315080011E001D15A7070471000FCE7C04688040020F9
S315080011F010B5FFF78DFF10BD0D4885460D480E4901
S315080012000E4A002302E0D458C4500433C4188C4252
S31508001210F9D30B4A0B4C002301E013600432A242B7
S31508001220FBD3FFF7ADFB02F095FAFFF777FAFEE777
S3150800123000100020000000200C000020303A0008B2
S3150800124010000020E8040020FEE7000070B5050045
S31508001250FA200D4B80001978FEF76AFF0B4B010048
S315080012601868FEF765FF00F083FB04000120002CD8
S3150800127009D1032D07D802382200290000F042FBC5
S315080012802000034B1D6070BD0600002000000020F2
S31508001290080000201023064A10B5116803200B43E6
S315080012A01360FFF7D3FFFFF7EFFA002010BDC04623
S315080012B000200240014B18687047C046C004002051
S315080012C00321036870B59A6804000A40012A01D010
S315080012D0002070BD1968114202D1DA681204F7D5E8
S315080012E005229D681540012D1ED19968033A0A43C7
S315080012F09A6003221A60FFF7DDFF060023689B68E1
S315080013002B42E5D0FFF7D6FF801B0228F6D92368C3
S315080013109B682B42F2D01023A26B01201343A363D0
S31508001320E36B1D43E563D4E710230120A26B134347
S31508001330A363E36B0343E363CBE70000002373B5C2
S3150800134003210193036804009A680A40012A07D119
S315080013501968114201D0002076BDDA681204FAD461
S3150800136099681B4A114208D010230120A26B134327
S31508001370A363E36B0343E363EEE7012299680A4339
S315080013809A60144B14491868FEF7D2FE0190019B27
S31508001390002B19D1FFF78EFF0125060023681B686D
S315080013A02B42D8D1FFF786FF801B0228F6D923687F
S315080013B01B682B42F2D11023A26B01201343A363AF
S315080013C0E36B1D43E563C7E7019B013B0193DEE73A
S315080013D0170000800000002040420F000422036826
S315080013E070B599680400114201D1002070BD996852
S315080013F0114206D09A68920703D4102299680A43C4
S315080014009A60FFF757FF0426050023689B68334256
S31508001410EBD0FFF74FFF401B0228F6D923689B68DD
S315080014203342F2D010230120A26B1343A363E36B6C
S315080014300343E363DAE70000F8B504000120002C53
S3150800144000D180E0A36B002B06D122003432E3637F
S3150800145020001370FFF728F8A36BDB0600D587E09A
S3150800146023680422996808001040114200D07FE0E2
S31508001470A26B4249114002220A430321A2639A68D9
S315080014800A40012A05D1196811420ED1DA681204F8
S315080014900BD41821DA688A43A1680A43DA60196905
S315080014A062688900890811431961DA6834490A4073
S315080014B0DA60A26A267E571E7A1E9741617EE26826
S315080014C0C903B6030E43A57E1643226969033F0383
S315080014D00E43022A00D10420621DD27FE17E52000B
S315080014E032433A430243012904D1002D2CD18021ED
S315080014F049020A43C220E169FF30814202D0206ACC
S3150800150001430A438020D96840051143D960E16A3E
S31508001510814202D0481E062807D80725586929405F
S31508001520A8435861586901435961DB6815490B405E
S31508001530934211D100200322E063A36B93431A0060
S3150800154001231343A363F8BD2020A56B2843A0639A
S31508001550E06B0143E163CDE71222A36B01209343BD
S315080015601A0010231343A363E36B0343E363EAE719
S315080015701023A26B01201343A363E4E7FDFEFFFFDC
S315080015801902FEFFE7FF3F83F7B5036804009B686F
S315080015900E00022001925B0730D4270034373B78CF
S315080015A0012B2BD001233B70637E012B27D1A36B24
S315080015B0164A00251A4080235B001343A363E5639C
S315080015C03D70206B124B21688362124BC362124B2B
S315080015D003631C230B604A680C3B13434B600123CF
S315080015E0CA681343CB603200019B403100F00CFA05
S315080015F004232800226891680B439360FEBD2000EF
S31508001600FFF79CFE0028D2D0F8E7C046FEF0FFFFA1
S31508001610991600080B17000819170008F8B50600F0
S315080016203436337805000224012B24D0012737707D
S31508001630FFF7D4FE041E1CD12A68286BD368BB4367
S31508001640D360831CDB7F022B07D100F01BFA041E34
S3150800165003D04023AA6B1343AB6310212A682800E2
S3150800166053688B435360002C07D1FFF729FE041EED
S3150800167006D0002333702000F8BDFFF721FEF8E7F7
S31508001680AB6B034A1A4001231343AB63F1E7C04629
S31508001690FEFEFFFF704700005022436A10B5996BA3
S315080016A011422AD1996BB132FF320A43C0219A639B
S315080016B01A680901D068084212D1997E00290FD10B
S315080016C0116809070CD5916849070DD40C20516893
S315080016D0814351609A6B0B49114001220A439A6370
S315080016E01800FFF7D7FF10BD2022996B0A439A63AB
S315080016F00122D96B0A43DA63F2E71B6B1B6B984727
S31508001700F1E7C046FEFEFFFF704710B5406AFFF7D7
S31508001710FBFF10BD704770474023406A10B5826BC7
S31508001720134383630423C26B1343C363FFF7F3FFB7
S3150800173010BD00000422036870B519680400114240
S3150800174002D05968114206D108221968114228D0D8
S315080017505968114225D0A26BD20604D48022A16B07
S3150800176092000A43A263C022D9681201114212D11B
S31508001770A27E002A0FD11A6812070CD59A6852075A
S315080017803CD40C215A688A435A60A36B204A1A40F3
S3150800179001231343A3632000FFF77CFF0C22236871
S315080017A01A60802523681A682A420CD05B682B4287
S315080017B009D08023A26B5B021343A3632000FFF7C3
S315080017C0A9FF23681D60102223681968114214D0E6
S315080017D05968114211D0A26A012A02D0DA68D207E2
S315080017E008D50222E16B20000A43E26310221A6040
S315080017F0FFF791FF102223681A6070BD2023A26BA1
S315080018001343A3630123E26B1343E363C3E7C046B1
S31508001810FEFEFFFFF0B50023040085B003933434C1
S3150800182023780200C66A0220012B2FD001382070C7
S31508001830136804279D68AC463D40019565463D42C0
S3150800184051D10F682A4D3A00AC464D68B840103A57
S31508001850654537D09D6A28439862802040058642B0
S315080018600FD0013E062E0CD907205D698968054010
S31508001870A94206D05D69014085435D615D692943DA
S315080018805961012A04D900200023237005B0F0BD50
S31508001890184A80211368102F12D0C9030B4313600E
S315080018A0102FF0D1144B15491868FEF741FC0A238E
S315080018B043430393039B002BE5D0039B013BF8E7C7
S315080018C00904EBE7996A81439962012ADBD85342F6
S315080018D05A4152420749920D9305094A08689B18CE
S315080018E003400B60CFE72023916B0B439363CBE751
S315080018F001100000082701400000002040420F00A8
S31508001900FFFFBFFF30B5FF2503242A000440E4008B
S31508001910A24089012940D243A140C3B200280ADB6C
S31508001920C0240B4B80088000C018A40003591A4035
S315080019301143015130BD0F200340083B05489B0861
S315080019409B001B18D86902401143D961F2E7C046CB
S3150800195000E100E000ED00E0002805DB1F23184049
S315080019601E3B8340014A13607047C04600E100E011
S315080019708022431E5204012093420DD2C021074AF9
S3150800198007485360036A09061B021B0A0B430362D6
S3150800199000200723906013607047C04610E000E0FF
S315080019A000ED00E070B504000120002C24D00223CD
S315080019B0A51CEB772068114B0268A1681A4063687A
S315080019C00B43E1680B4321690B4361690B43A1692A
S315080019D00B43E1690B4313430360094B1421C018F9
S315080019E0FEF7A6FB074B80002064E3630020012373
S315080019F0A063E418EB77E07770BDC0460FC0FFFF21
S31508001A00F8FFFDBF00000240F7B5451C0193EB7FC8
S31508001A1004000220012B27D001232718EB77FB7F30
S31508001A2000269C466046DBB2012828D10130F877AB
S31508001A302068A6630568266C9D43B3400560E56B80
S31508001A406B60019B43606368102B0ED18260C16096
S31508001A50E36A0268002B0BD00E23134303600123AD
S31508001A600268134303600020FEBD8160C260EFE791
S31508001A700A2313430422036003689343EEE7022014
S31508001A80EE77F1E730B5851CEB7F441C022B05D0B9
S31508001A900423836300230120E37730BD0E21036806
S31508001AA01A688A431A600122196891431960016C01
S31508001AB0C36B1000884058600020EA77E077ECE7AF
S31508001AC070B5841CE37F022B04D004238363033B95
S31508001AD0180070BD0E210368056C1A688A431A60DF
S31508001AE001221968914319601100A940C36B596016
S31508001AF0E27700248318DC77426B1300A242E7D012
S31508001B0090472300E4E7F8B504273E00016CC26B52
S31508001B108E40156803681C6835420DD03C420BD0D0
S31508001B201968890602D41968B9431960C36A5660E8
S31508001B30002B19D0984717E002273E008E40354201
S31508001B4013D03C4211D01968890606D40A241968AC
S31508001B50A14319600121C319D97756600022431C95
S31508001B60DA77836A9342E5D1F8BD082637008F40B5
S31508001B703D42F9D03442F7D00E251C68AC431C60B0
S31508001B8001231C008C405460821C8363D377002297
S31508001B90C318DA77036BE5E70230C07FC0B2704737
S31508001BA0806B70470C4A1021D06830B503000B4093
S31508001BB0084205D002230948C4692343C3610B00C0
S31508001BC00420D168014205D00121044C0343E5698C
S31508001BD02943E161D36030BD00200240C8040020DB
S31508001BE0064B00201A69120606D5054A5A60054AA8
S31508001BF05A6018690006C00F7047C04600200240A8
S31508001C0023016745AB89EFCD8023034A002011697C
S31508001C100B4313617047C0460020024070B50400AC
S31508001C20FFF748FB01260500104BDA68324211D14E
S31508001C302022D968114200D0DA60D968102208003B
S31508001C401040114202D1DB685B0708D5FFF7AAFFEF
S31508001C50012004E0621CE8D0002C01D1032070BDED
S31508001C60FFF728FB401BA042DED9F7E70020024019
S31508001C70F0B585B003931C4B019102921A7E0400BD
S31508001C800220012A2ED0012218481A76FFF7C6FF2D
S31508001C90002824D12600012C02D0022C00D00426CC
S31508001CA00024029803992201FEF7B8FB00220127B7
S31508001CB00D4B0F4DDA612B69019A3B432B6163008B
S31508001CC09B1880B218800948FFF7A8FF2B69BB4309
S31508001CD02B61002803D1E419E3B29E42E1D8002221
S31508001CE0014B1A7605B0F0BDC804002050C30000A9
S31508001CF0002002400022064BDA61064B04321969BD
S31508001D000A431A61402219690A431A617047C04694
S31508001D10C8040020002002400022064BDA61064B68
S31508001D20023219690A431A614022586119690A433D
S31508001D301A617047C804002000200240F8B5214FF8
S31508001D4004003B7E0E000220012B0CD001233B76BB
S31508001D5023681D48012B12D1FFF760FF002803D026
S31508001D60012000233B76F8BDFFF7C4FF1648FFF7AE
S31508001D7055FF0421154A13698B431361F1E7FFF7F1
S31508001D804DFF0028ECD101235B42336065680130C2
S31508001D90A36862689B029B18AB42E2D92800FFF74A
S31508001DA0BBFF0948FFF73AFF0221084A13698B432C
S31508001DB01361002801D03560D3E78023DB00ED18D6
S31508001DC0E6E7C046C804002050C3000000200240D1
S31508001DD00023F0B587B00A681400DC4001D107B0CB
S31508001DE0F0BD012514009D402C4001942A4200D1E3
S31508001DF095E04A685E00944603226446224003241E
S31508001E00B440E4430294541E012C2AD88768029CE5
S31508001E102740CC68B4403C43846044680127AC43FF
S31508001E202500644624093C409C402C434460C56810
S31508001E30029C25408C68B4402C43C460022A12D107
S31508001E40DC080725A4000419276A03940F241D40FB
S31508001E50AD00AC40A7430C69AC402743039C2762FE
S31508001E6001E0032AE3D10468029DB24025402C0014
S31508001E7014430460C0246246A40222424FD00125BE
S31508001E80284A90279469FF052C43946192699C0817
S31508001E902A400592059A244AA400A4180F2202355E
S31508001EA01D40AD00AA40A66896430022B8420CD051
S31508001EB01E4F0132B84208D01D4F0132B84204D035
S31508001EC01C4F0132B84200D00232AA40674632435C
S31508001ED0A260194A019C1668019DE4433543FF0335
S31508001EE001D435002540674615605668019D35437F
S31508001EF0BF0301D435002540674655609668019DA5
S31508001F003543FF0201D43500254067469560D568FC
S31508001F10019E2E43BF0201D425402E00D660013310
S31508001F2059E7C0460010024000000140000400487E
S31508001F3000080048000C00480004014000690840F9
S31508001F40431E9841C0B27047002A01D0816170478C
S31508001F508162FCE7426913000B401B049143194355
S31508001F6081617047044B10B55A69104202D0586116
S31508001F70FFF73CF810BDC0460004014070B50400E8
S31508001F800120002C17D02368124A07251A60124A26
S31508001F901A6062685A60A2689A60FFF78BF90600B1
S31508001FA02368DA68100028402A4205D11969E268D0
S31508001FB091420CD01A6170BDFFF77CF9801B272867
S31508001FC0EED92368DB682B42EAD00320F3E7034AFD
S31508001FD01A60F0E7CCCC000055550000AAAA00000C
S31508001FE00368024A00201A607047C046AAAA000081
S31508001FF0F0B5040085B0002845D00368DB072FD468
S3150800200023689B0700D581E023681B0700D5BCE041
S3150800201023685B0700D5DFE02368DB061AD562690B
S315080020200423B54D012A00D04AE1696B02270B4308
S315080020306B636B6B1A436A63FFF73CF906006B6BBD
S315080020403B4200D135E1F8216A6BA3698A43DB007C
S3150800205013436B63236A002B00D059E100202AE062
S315080020600C21A54D6A680A40042A06D06B680B4005
S31508002070082B0AD16B68DB0307D52B689B03BFD5F2
S315080020806368002BBCD1012015E06368012B14D1CD
S3150800209080232A685B0213432B60FFF70BF980271E
S315080020A00600BF022B683B42AAD1FFF703F9801B43
S315080020B06428F7D9032005B0F0BD002B16D12B688C
S315080020C08E4A802713402B602B688D4ABF02134027
S315080020D02B60FFF7EFF806002B683B4200D18FE72D
S315080020E0FFF7E8F8801B6428F6D9E3E7052B05D146
S315080020F080232A68DB0213432B60C9E72B687F4AD3
S3150800210013402B602B687E4A1340C5E70C227A4D94
S315080021106B68134206D06B681340082B10D16B68A6
S31508002120DB030DD42B689B0702D5E368012BAAD1E4
S31508002130F8212A6823698A43DB0013432B6063E787
S31508002140E2680123002A0FD02A68022713432B606E
S31508002150FFF7B0F806002B683B42E9D1FFF7AAF86B
S31508002160801B0228F7D9A5E72A6802279A432A601E
S31508002170FFF7A0F806002B683B4200D144E7FFF7BB
S3150800218099F8801B0228F6D994E7E26901235A4D8B
S31508002190002A10D06A6A022713436B62FFF78AF88F
S315080021A006006B6A3B4200D032E7FFF783F8801BD4
S315080021B00228F6D97EE76A6A02279A436A62FFF717
S315080021C079F806006B6A3B4200D121E7FFF772F8FF
S315080021D0801B0228F6D96DE780220021464D52055C
S315080021E0EB690091134208D1EB691343EB61EB6984
S315080021F013400393039B012300938027414E7F00DE
S3150800220033683B4206D0A368012B13D12A6A1343CD
S315080022102B6230E033683B433360FFF74BF801909D
S3150800222033683B42EFD1FFF745F8019BC01A642893
S31508002230F6D93FE70122002B14D12B6A02279343D4
S315080022402B622B6A033293432B62FFF733F806009F
S315080022502B6A3B4216D0FFF72DF82B4B801B984272
S31508002260F6D927E7052B16D1296A013B0B432B62C2
S315080022702B6A1A432A62FFF71DF8022706002B6A03
S315080022803B420FD0009B012B00D0C5E6EB691F4AE5
S315080022901340EB61C0E62B6A934304222B622B6A38
S315080022A09343B5E7FFF706F8174B801B9842E6D924
S315080022B000E7FEF7FFFF801B022800D8BFE6F9E615
S315080022C0053203D16A6B9A436A63BCE66A6B0227D6
S315080022D0134301226B636B6B93436B63FEF7EAFF51
S315080022E006006B6B3B4200D1B4E6FEF7E3FF801BAA
S315080022F00228F6D9DEE6C04600100240FFFFFEFFC0
S31508002300FFFFFBFF0070004088130000FFFFFFEF90
S315080023100C21344D6A680A40082A47D0324A022BF3
S3150800232032D12B68802713402B60FEF7C3FF0600C7
S31508002330BF042B683B4221D10F22EB6A80269343C8
S31508002340E26AB6041343EB62616AA36A6A680B43DE
S3150800235026490A4013436B6080232A685B041343AB
S315080023602B60FEF7A7FF04002B68334200D075E602
S31508002370FEF7A0FF001B0228F6D99BE6FEF79AFF98
S31508002380801B0228D5D995E62B68802613402B603A
S31508002390FEF790FF0400B6042B68334200D15DE6D1
S315080023A0FEF788FF001B0228F6D983E61800012BE2
S315080023B000D180E680216B68606A4902EA6A1940A2
S315080023C0814200D05FE60F210A40E16A8A4200D0C6
S315080023D059E6F02292031340A26A934200D13DE6E1
S315080023E051E6C04600100240FFFFFFFEFFFFC2FF96
S315080023F070B588B010221249684604AD01F0CEF9CE
S31508002400102228000F4901F0C9F90C220E4E7368F4
S315080024101A40082A11D10F206A46990C0140545CCB
S31508002420F26A0240A95CDB0305D50848FDF780FE81
S31508002430604308B070BD0648FAE70448F9E7C046A5
S31508002440003A0008113A00080010024000127A000B
S3150800245000093D00F7B504000E00002801D101204F
S31508002460FEBD0122374D2B6813408B421CD32168D1
S315080024708B0722D4CB072FD401232A681A40B242ED
S3150800248051D82368304D5B0754D4FFF7B1FF6B680A
S315080024902E4A1B061B0FD35CD8402D4B1860032011
S315080024A0FEF7D4FE0020DBE72B6893430B432B6033
S315080024B02B6813408B42D2D1D9E7234A4B0704D560
S315080024C0E0235068DB0003435360F02053688343DE
S315080024D0A06803435360CDE71B4F62683B68012A37
S315080024E019D19B03BBD503217B688B4313437B60C0
S315080024F0FEF7E0FE01900C237A681A4063689B0099
S315080025009A42B9D0FEF7D6FE019BC01A114B9842E3
S31508002510F1D90320A4E7022A02D19B01E3D49EE75E
S315080025209B07E0D49BE72A689A432A602A681A42DE
S31508002530A7D094E76B68084A1340E26813436B60B8
S31508002540A3E7C0460020024000100240D837000822
S315080025500000002088130000FFF8FFFF044B054A1F
S315080025605B685B055B0FD35C034A1068D84070470D
S3150800257000100240E837000800000020F0B50368A4
S31508002580050085B0DB032AD580220021384C520588
S31508002590E3690091134208D1E3691343E361E369F0
S315080025A013400393039B012300938027314E7F003A
S315080025B033683B4228D0226AC02311009B002E4E66
S315080025C019401A4232D1236A1E406B681E43009B8B
S315080025D02662012B03D1E369284A1340E3612A687E
S315080025E0D30706D5032022490B6B8343A868034308
S315080025F00B630020930617D510211D4A136B8B43D6
S31508002600E9680B4313630FE033683B433360FEF717
S3150800261051FE019033683B42CDD1FEF74BFE019B3C
S31508002620C01A6428F6D9032005B0F0BD6A681340BD
S315080026308B42C8D08023226A206A11005B020343BA
S315080026402362236A0E483140034023622162D3077E
S31508002650B9D5FEF72FFE07000222236A1342B2D12C
S31508002660FEF728FE074BC01B9842F5D9DBE7C046A4
S315080026700010024000700040FFFCFFFFFFFFFFEF65
S31508002680FFFFFEFF881300000122036A70B593431B
S315080026900362036A44688569723295430A6815437A
S315080026A0022293438A681343114A904205D0114E79
S315080026B0B04202D0104EB04213D10826B343CE68BA
S315080026C033430426B343904205D00A4A904202D0C7
S315080026D0094A904205D1094A8E6922404C69344319
S315080026E014434A68446085614263036270BDC0460C
S315080026F0002C01400044014000480140FFFCFFFF58
S3150800270070B57325036A164A13400362036A426862
S31508002710C469AC430D682C43124D2B408D682D02BD
S315080027202B43114DA8420ED1104D1D40CB681B02FC
S315080027302B430F4D2B400F4D4E6915408A69324386
S3150800274012012A4305E00C4DA842F4D00B4DA842CD
S31508002750F1D042604A68C461C263036270BDC04674
S31508002760FFFEFFFFFFFDFFFF002C0140FFF7FFFF05
S31508002770FFFBFFFFFFCFFFFF004401400048014079
S31508002780036A124A30B513400362026A104C436862
S31508002790C56925400C68240225430E4C22408C68E6
S315080027A0240322430C4CA04205D00C4CA04202D074
S315080027B00B4CA04204D10B4C23404C69A401234383
S315080027C043604B68C5610364026230BDFFEFFFFFDB
S315080027D0FF8CFFFFFFDFFFFF002C01400044014094
S315080027E000480140FFBFFFFF0200030001203D3201
S315080027F01178814215D1022111701B68DA680243EB
S31508002800DA600B4A934202D00A4A93420AD1072158
S315080028109A6800200A40062A03D0012219680A434A
S315080028201A6070471A68104318600020F9E7C04616
S31508002830002C0140000400407047704770477047FD
S31508002840704770470222036810B5196904001142DF
S315080028500ED0D96811420BD0053A1A6104320277B4
S315080028609B699B0700D179E0FFF7E9FF00232377EF
S31508002870042223681969114210D0D96811420DD073
S31508002880093A1A61073222779A69C0239B00200009
S315080028901A4269D0FFF7D3FF00232377082223685B
S315080028A0196911420ED0D96811420BD0113A1A6132
S315080028B00D322277DB6920009B075BD0FFF7BFFF4D
S315080028C000232377102223681969114210D0D9688A
S315080028D011420DD0213A1A6119322277DA69C023DA
S315080028E09B0020001A424BD0FFF7A9FF002323774D
S315080028F0012223681969114207D0D968114204D008
S31508002900033A20001A61FFF798FF802223681969A5
S31508002910114208D0D968114205D0023AFF3A200080
S315080029201A6100F0DCF9402223681969114207D0C0
S31508002930D968114204D0813A20001A61FFF781FF55
S31508002940202223681969114207D0D968114204D098
S31508002950413A20001A6100F0C1F910BDFFF76EFF79
S315080029602000FFF76DFF81E7FFF768FF2000FFF7FC
S3150800297067FF91E7FFF762FF2000FFF761FF9FE718
S31508002980FFF75CFF2000FFF75BFFAFE7194A10B5BA
S315080029900368904202D0184CA04208D17024A34381
S315080029A04C68234390420BD0134CA04208D0134CDA
S315080029B0A04205D0124CA04202D0124CA04203D12C
S315080029C0114C2340CC6823438024A3434C692343FA
S315080029D003608B68C3620B688362904205D0084B1C
S315080029E0984202D0074B984201D10B690363012331
S315080029F0436110BD002C0140000400400020004047
S31508002A000044014000480140FFFCFFFF70B5040088
S31508002A100120002C21D025003D352B78DAB2002B79
S31508002A2005D123003C3320001A70FDF7ABFF0223C3
S31508002A302B702068211DFFF7A9FF22000123002023
S31508002A40463213704534083A137053709370D37036
S31508002A5013715371937123702B7070BD70B5040098
S31508002A600120002C21D025003D352B78DAB2002B29
S31508002A7005D123003C3320001A70FFF7DDFE022340
S31508002A802B702068211DFFF781FF220001230020FB
S31508002A90463213704534083A137053709370D370E6
S31508002AA013715371937123702B7070BD1022036AD2
S31508002AB070B593430362026A154C436885692540DD
S31508002AC00C68240225432024A2438C68240122434F
S31508002AD0104CA0420FD18024A2431400CA681201E8
S31508002AE022434024A2430C4E4C691E408B69234363
S31508002AF09B00334305E0094CA042F4D0084CA042A1
S31508002B00F1D043604B6885618363026270BDC0463D
S31508002B10FF8CFFFF002C0140FFF3FFFF004401403C
S31508002B2000480140F8B507003C373B7804000E0022
S31508002B3015000220012B0AD001383870082A3DD02A
S31508002B4006D8002A17D0042A27D000233B70F8BDE0
S31508002B500C2AFAD12068FFF713FE80222368120197
S31508002B60D9690A43DA61DA691C490A40DA613269C5
S31508002B70D96912022FE02068FFF786FD082223682C
S31508002B8099690A4304219A619A698A439A619A69FA
S31508002B9031690A439A610020D7E72068FFF786FF64
S31508002BA080222368120199690A439A619A690B4936
S31508002BB00A409A61326999691202EAE72068FFF7C2
S31508002BC09FFD04212368DA691543DD61DA698A43C2
S31508002BD0DA61DA6931690A43DA61DCE7FFFBFFFF8C
S31508002BE01F2310B5012419408C408A40036AA34369
S31508002BF00362036A1A43026210BD000010B504009E
S31508002C00002906D1020001203E321378834238D0CB
S31508002C1010BD030004292ED13F331B780120013B48
S31508002C205A1E9341DBB2002BF2D10223220004295B
S31508002C302DD13F3213702268D3680B43D3602068C6
S31508002C400122FFF7CDFF23681E498B422CD01E4A6E
S31508002C50934229D01D4A934226D01D4A93422BD12E
S31508002C6007219A6800200A40062AD1D0012219684D
S31508002C700A431A60CCE7082901D14033CDE741332E
S31508002C80CBE7022313702268D0680343D6E70829E6
S31508002C9001D14032CEE74132012013700C29B7D159
S31508002CA022681023D068F0E78022586C120202438B
S31508002CB05A648B42D1D1D3E70122196800200A430E
S31508002CC01A60A5E7002C0140004401400048014075
S31508002CD00004004010B5FFF791FF10BD704770471C
S31508002CE030B5EFF31084012282F310880168124D83
S31508002CF00B682B400B6084F31088EFF3108482F383
S31508002D00108801688B6893438B6084F31088036E80
S31508002D1093420AD1EFF3108183F3108810240268D6
S31508002D201368A343136081F310882023C367002325
S31508002D300366436630BDC046DFFEFFFFF7B51300E6
S31508002D40826F04000220202A3AD10138002937D0A0
S31508002D50002B35D08022A0685201904206D1226904
S31508002D60002A03D101321000114229D125007435F9
S31508002D702A780220012A23D001222A702200503202
S31508002D80E1640026138053802122E06E271DFE672A
S31508002D90A267B04215D0226846630192124A82623F
S31508002DA0124AC262124A0263019A2832FEF72CFEC0
S31508002DB0B04206D010230120FB67DB182E70A367EC
S31508002DC0FEBD4022002023681A622870EFF31081A6
S31508002DD0012383F3108822687F3394682343936022
S31508002DE081F31088ECE7C046A92E0008F52E0008E6
S31508002DF0052F00088021026870B5836FC56F926839
S31508002E0004000A422BD0212B29D1EFF31080203B56
S31508002E1083F31088226893688B43936080F3108845
S31508002E20E06E00280DD0FEF72DFE002809D0E06ED2
S31508002E30FEF7B6FE202804D110230434E3671D38B4
S31508002E4070BDEFF31081012383F31088C020226838
S31508002E5013688343136081F310882023A3674021F6
S31508002E60236800209B680B42EAD0222DE8D1EFF3B5
S31508002E701080012383F31088226893688B4393603C
S31508002E8080F31088206F002808D0FEF7FBFD002885
S31508002E9004D0206FFEF784FE2028CDD02000FFF74F
S31508002EA01FFF0020CCE7704703009B6970B5406A96
S31508002EB0202B1BD00300002252331A80EFF3108414
S31508002EC0013282F31088802501688B68AB438B60DA
S31508002ED084F31088EFF3108182F310884023026888
S31508002EE010680343136081F3108870BDFFF7DBFF9A
S31508002EF0FBE7704710B5406AFFF7FBFF10BD704748
S31508002F007047704770B5446A2268A36FE16F92688C
S31508002F10120613D5212B11D12300002252331A8011
S31508002F20EFF31080012383F31088C0252268136805
S31508002F30AB43136080F310882023A36723689B683C
S31508002F405B0608D5222906D1230000225A33200021
S31508002F501A80FFF7C5FE1023221DD16F20000B43F0
S31508002F60D367FFF7CEFF70BD406A0023020010B595
S31508002F705A321380083A1380FFF7C3FF10BD704713
S31508002F800168F8B5CB699F4D040008688A682B422A
S31508002F900BD12022134200D17EE0104200D17BE003
S31508002FA0636E2000002B6DD16DE00126964D3240F0
S31508002FB00540154300D16FE0251D334205D0C705EE
S31508002FC003D50E62EF6F3E43EE670226334206D004
S31508002FD0002A04D00E62EF6FB6193E43EE67042648
S31508002FE0334206D0002A04D00E62EF6F023E3E43FB
S31508002FF0EE670826334207D0202707403A4303D016
S315080030000E62EA6F1643EE6780221201134206D05B
S31508003010460104D50A622022E96F0A43EA67EA6F85
S31508003020002A30D02022134206D0104204D0636E04
S31508003030002B01D0200098472268EB6F402796683E
S3150800304028223E40134020001E4321D0FFF748FEA9
S3150800305023689B683B4217D0EFF31081012383F363
S31508003060108822689368BB43936081F31088206FA9
S31508003070002809D0654B4363FEF722FD002802D0DD
S31508003080206F436B9847F8BD2000FFF73AFFFAE731
S31508003090FFF737FFEE67F6E7226E012A00D090E0C9
S315080030A010252B4200D18CE0284200D189E00D6220
S315080030B08B684021180008400B424CD0206F0368EB
S315080030C05B689BB2002BDED02600583637889F42B5
S315080030D0D9D927005A373B808369202B31D0EFF3A3
S315080030E0108782F310882068494D03682B400360D7
S315080030F087F31088EFF3108782F3108820688368B7
S315080031009343836087F31088EFF3108782F3108860
S31508003110206883688B43836087F310882023E367DE
S3150800312000232366EFF3108182F310882268123594
S315080031301368FF35AB43136081F31088206FFEF7E1
S31508003140A1FC23005A331B883188C91A89B220008A
S31508003150FFF715FF97E726005A36338831889BB262
S31508003160002900D18FE7210058310988C91A89B288
S31508003170002900D187E7EFF3108782F310882668C5
S31508003180244D33682B40336087F31088EFF310879C
S3150800319082F310882668B3689343B36087F3108870
S315080031A020236066E3672066EFF3108082F31088B9
S315080031B0226832351368FF35AB43136080F31088F5
S315080031C0C5E78022134203D0104201D0A36EE8E679
S315080031D04022134200D156E7104200D153E7EFF3DD
S315080031E01080012383F3108821680B6893430B60D2
S315080031F080F310882023A36700232000A366FFF727
S3150800320052FE40E70F08000020010004692F00085D
S31508003210FFFEFFFFDFFEFFFF406A10B5036E012BBE
S3150800322006D10300583319884908FFF7A8FE10BDD0
S31508003230FFF766FEFBE7000003009B6970B5406A6E
S31508003240202B34D0030000225A331A80EFF310845F
S31508003250012383F3108801681B4D0A682A400A6017
S3150800326084F31088EFF3108483F3108801688A6862
S315080032709A438A6084F31088EFF3108183F31088E9
S31508003280402402689368A343936081F3108820233F
S31508003290C367036E012B0AD1EFF3108183F31088FD
S315080032A00268303C1368A343136081F31088036EE9
S315080032B0012B05D1030058331988FFF760FE70BD4E
S315080032C0FFF71DFEFBE7C046FFFEFFFF70B50400D3
S315080032D02569A26801682A436569C3692A4308689B
S315080032E0394D1A43284002430A604A683748256A16
S315080032F00240E06802434A60A26988682A43344D5E
S31508003300284002438A600321324A126B0A40802110
S31508003310013A0902022A4CD82F48805C8B4224D1F4
S31508003320082817D8FCF7FAFE4716081605161616C3
S315080033300900FFF75DF840E0284B580063686168AC
S315080033405B08C018FCF7F4FE254982B2103A03045C
S315080033508A4201D9012033E00F221B03904380B231
S3150800336022685B0F1843D06029E00828F2D8FCF7DA
S31508003370CBFE16F11EF11BF1F1F1050080200002CB
S31508003380636861685B081818FCF7D2FE80B2020011
S31508003390134B103A9A42DDD82368D8600FE0FFF73E
S315080033A0DDF800280BD0EBE7FFF722F8F9E70B4822
S315080033B0E6E78B42F3D1FFF7D1F8031EBDD1002013
S315080033C000236366A36670BDF369FFFFFFCFFFFFA7
S315080033D0FFF4FFFF00100240223A000800127A00AC
S315080033E0EFFF0000436A30B5DA0706D50168284CB6
S315080033F04A682240846A22434A609A0706D50168C9
S31508003400244C4A682240C46A22434A605A0706D5B1
S315080034100168214C4A682240046B22434A601A0715
S3150800342006D501681D4C4A682240446B22434A600F
S31508003430DA0606D501681A4C8A682240846B22434C
S315080034408A609A0606D50168164C8A682240C46BBB
S3150800345022438A605A0610D50168134D4A68046CDF
S315080034602A4022434A6080225203944205D14A6880
S315080034700E4C2240446C22434A601B0606D502685D
S315080034800B4953680B40816C0B43536030BDC046F3
S31508003490FFFFFDFFFFFFFEFFFFFFFBFFFF7FFFFFB5
S315080034A0FFEFFFFFFFDFFFFFFFFFEFFFFFFF9FFFBE
S315080034B0FFFFF7FFF7B5802704000D0016000193FC
S315080034C03F012268D3692B405B1B59424B41B342EB
S315080034D001D0002028E0089B0133F3D0FDF7EAFE6F
S315080034E0019BC01A089B984201D8002B1DD1EFF307
S315080034F01080012282F3108821681E4D0B682B402C
S315080035000B6080F31088EFF3108082F3108821682F
S315080035108B6893438B6080F310882023A367E36747
S315080035200023032074342370FEBD042123681A681F
S315080035300A42C6D0DA693A42C3D01F62EFF3108056
S31508003540012282F3108821680A4D0B682B400B6014
S3150800355080F31088EFF3108082F3108821688B6857
S3150800356093438B6080F310882023221DA367E367AB
S31508003570D367D5E75FFEFFFF73B500260400031D7A
S31508003580DE67FDF797FE236805001B681B0716D440
S3150800359023681B685B070AD580210F4B002200931E
S315080035A020002B00C903FFF785FF002812D120232E
S315080035B00020A367E3672066743420700BE080213F
S315080035C0054B32000093890303002000FFF772FFC2
S315080035D00028DDD0032076BDFFFFFF0110B5041ECD
S315080035E001D1012010BD836F002B04D10200743273
S315080035F01370FDF75FFA242301212268A367136875
S3150800360020008B431360FFF761FE0128E9D0636A47
S31508003610002B02D02000FFF7E5FE236807495A6809
S3150800362020000A4008215A609A688A439A60012253
S3150800363019680A431A60FFF79FFFD3E7FFF7FFFFF2
S31508003640F8B51300020004005832416500251380BE
S3150800365022222600071DFD67C267006F7436A8423E
S3150800366016D01E4A456382621D4AC2621D4A02631B
S315080036702268243294460A006146FEF7C5F9A84234
S3150800368006D010230120FB67DB183570E367F8BD09
S3150800369000203070EFF31085012383F31088802211
S315080036A0216852000E6832430A6085F31088EFF3EA
S315080036B0108583F3108821688A681A438A6085F31F
S315080036C01088EFF3108183F3108822683F339468DB
S315080036D02343936081F31088D9E7C046393200083E
S315080036E019320008052F000870B5C46F0223202C74
S315080036F02DD1013B00292AD0002A28D080238468AE
S315080037005B019C4206D10369002B03D101242300E7
S3150800371021421CD10400743425780223012D16D0C9
S31508003720013B2370002404660468646824020BD5F0
S31508003730EFF3108583F3108880230468DB0426687A
S315080037403343236085F31088FFF77AFF03001800D8
S3150800375070BD000070B500260C4D0D4C641BA410FE
S31508003760A64209D1002600F02BF80A4D0A4C641B24
S31508003770A410A64205D170BDB300EB589847013690
S31508003780EEE7B300EB5898470136F2E7283A000807
S31508003790283A0008283A00082C3A0008002310B5F1
S315080037A09A4200D110BDCC5CC4540133F8E703003B
S315080037B08218934200D1704719700133F9E7000067
S315080037C0F8B5C046F8BC08BC9E467047F8B5C04672
S30D080037D0F8BC08BC9E467047D0
S315080037D800000000000000000102030406070809AB
S315080037E800000000010203044443452D32333032F9
S315080037F82D56345F48414C0000C1814001C08041C4
S3150800380801C0804100C1814001C0804100C181409A
S3150800381800C1814001C0804101C0804100C181408A
S3150800382800C1814001C0804100C1814001C080417A
S3150800383801C0804100C1814001C0804100C181406A
S3150800384800C1814001C0804100C1814001C080415A
S3150800385801C0804100C1814000C1814001C080414A
S3150800386801C0804100C1814001C0804100C181403A
S3150800387800C1814001C0804101C0804100C181402A
S3150800388800C1814001C0804100C1814001C080411A
S3150800389801C0804100C1814000C1814001C080410A
S315080038A801C0804100C1814001C0804100C18140FA
S315080038B800C1814001C0804100C1814001C08041EA
S315080038C801C0804100C1814001C0804100C18140DA
S315080038D800C1814001C0804101C0804100C18140CA
S315080038E800C1814001C0804100C1814001C08041BA
S315080038F801C0804100C1814000C0C101C30302C2A2
S31508003908C60607C705C5C404CC0C0DCD0FCFCE0E09
S315080039180ACACB0BC90908C8D81819D91BDBDA1A79
S315080039281EDEDF1FDD1D1CDC14D4D515D71716D6E9
S31508003938D21213D311D1D010F03031F133F3F23259
S3150800394836F6F737F53534F43CFCFD3DFF3F3EFEC9
S31508003958FA3A3BFB39F9F83828E8E929EB2B2AEA39
S31508003968EE2E2FEF2DEDEC2CE42425E527E7E626A9
S3150800397822E2E323E12120E0A06061A163A3A26219
S3150800398866A6A767A56564A46CACAD6DAF6F6EAE89
S31508003998AA6A6BAB69A9A86878B8B979BB7B7ABAF9
S315080039A8BE7E7FBF7DBDBC7CB47475B577B7B67669
S315080039B872B2B373B17170B05090915193535292D9
S315080039C896565797559594549C5C5D9D5F9F9E5E49
S315080039D85A9A9B5B99595898884849894B8B8A4AB9
S315080039E84E8E8F4F8D4D4C8C448485458747468629
S315080039F88242438341818040020304050607080979
S31508003A080A0B0C0D0E0F1010000102030405060719
S31508003A1808090A0B0C0D0E0F100004080200000016
S30908003A28E90000089B
S30908003A2CC1000008BF
S31108003A3000127A000101010004000000E9
S705080011F9E8
